:020000040000FA
:1000000007309F0083169F01003086008500831211
:100010003830532001305320033053200F30532009
:10002000803053208316F030860081138312EF3026
:10003000A50086000430A000A50C250886006B20D2
:1000400006080F38A100A109031D2928A00B1C28B0
:10005000172806080F38A400A409031D29288316B1
:10006000003086008312A50925080F39A500210854
:10007000F039A504250886001130A100A10321084C
:1000800073202502031D3E28210886001030210719
:1000900073208600A500003083160030860083128E
:1000A00025085F20122886006B20043085006B2015
:1000B000003085006B20043085006B20080086002E
:1000C0006B20063085006B20023085006B200630E7
:1000D00085006B2008003230A300A200A20B6E281E
:1000E000A30B6D280800820711341234143418341D
:1000F00021342234243428344134423444344834C2
:10010000813482348434883430343134323433347A
:100110003434353436343734383439344134423475
:080120004334443445344634F5
:02400E00293F48
:00000001FF
